:020000040000FA
:10000000000000002000052807296400A701C101A5
:10001000C114C310182800000000000000000000F8
:100020000730083018304730183022300D300000CB
:100030007D30DF000301DD00D3205A08A63A031902
:100040002C28B401B501A801C001C301D0011830AA
:10005000C700F83AC900C3170130B6000830D00015
:1000600022008C0021000C308C00230000308C001A
:10007000240008308C0021006A30990021000530EE
:100080009500270008309100920093012100003074
:10009000910020003530980097010530B7002810F6
:1000A0000C1928140830B30064000130DD009820DA
:1000B000DC1F68287F30DF05031968285F093E3997
:1000C000031968285F08663C031C68285F086928D4
:1000D0003D30B0000330DD0098205F08DC1F0530A4
:1000E000C200A3200530DD0098205F08DC1F00302F
:1000F000C400441BC3140730DD0098205F08DC1FD8
:100100000130C500A3200930DD0098205F08DC1B0A
:100110008A207229A100F839B800B4004017FD20E8
:100120005F080F39B700BA005F08C039C204FF2B5F
:10013000FD20DF00DC175F085A3A031DDC13DD0ADF
:10014000FD20DF00080045090339CA0003144A0DE9
:10015000421A0639CA00210095002000450D0639D3
:10016000421A013E03190138D300CB010314CB0D11
:10017000D30BB72808000930DD00A530CF2842088E
:10018000C0393A04DF000B30DD00D3203908DF002E
:10019000C01B5F150A30DD00D320DD035A30DF00BD
:1001A0005D08D3200800230091002000FD205F0699
:1001B000031908005F082300930094012000E22047
:1001C000F1200800640023001513951315158B13F7
:1001D00055309600AA30960095148B171511200003
:1001E000080023009518F1282000DC17C0105012D9
:1001F0000C12D0128C12640008005D0823009100DC
:1002000092011513951315141308200008008B1B79
:10021000072920000B1916210B1C09000B102700C1
:10022000FF3013069305200039210900FC30D0056A
:10023000C31D2529C311411B28290330C31CD00429
:10024000FC30C01CD00546082D29C315C11A1D2934
:100250000130C01B0230D004480895000B11C110BA
:10026000951FC114500822008C002000B1174111C5
:1002700008000C0828060839031D08000C08083976
:1002800003194829A811970C160CA600A7150800F9
:10029000A81596019701A919552927185429300D39
:1002A000AF002F0D0338AF000800451E0800AF0D4A
:1002B0000318080020306B21D016500822008C0053
:1002C000200060306B21D012500822008C002000EA
:1002D000080064003030AE00AE0B6C296400702959
:1002E00071290800A630DA00E8308B00B101A03097
:1002F000BF006400A7197322C11C832941198329F7
:10030000F121C9216400A719732240182226A719D8
:1003100073229329A81C9329A810B30B9329BA21FF
:1003200029120830B300BE0B7929BF0B7929310897
:100330009F3AFE39031DB829431DA3294311401FCD
:10034000A3293808B400C014311C401B7629C519F4
:10035000AF293408F8390319AF2946247629B401A6
:10036000C010A813A8124213C2130530B700762993
:10037000DA0100280C1DC529281808002814A81324
:10038000A812C014C01B022C072C281C080028101F
:10039000BF29C11241133508FE39C900031DD229F6
:1003A000C916C11604304906FC390319C90D49089C
:1003B000FF3CC9003509FE39C700F839031DE229A1
:1003C000C71641174708083C0318E8294715C71501
:1003D0004708FF3CC700C6004908C8003116411550
:1003E0000800C31AF529C3160800C312B60B08008B
:1003F0004319B4014B08B6000310A81E112A431A72
:10040000B60DC11B112AC117A81BB20B0800A813F7
:10041000A812441BC3143A08B7003808401BB400A4
:100420000800C113C31F1F2A3508403C031C1B2AA8
:100430000530B7001F2AC3133A08401BB700401409
:10044000C11C272AB30B272ABA210830B300B115E3
:100450003408D500C41D3C2A37080E3A03193C2A3B
:100460000310B60D031C362AF830B600A81A3C2A31
:10047000411A3C2A41160800411235085502031959
:100480000800031CFF3A3702031C492A5508B5002F
:10049000080035083402031C502A3708B507080045
:1004A0003708B5020800281228135C138C12A70124
:1004B00008002008FF3A2206031D0534A91700345E
:1004C0002108FF3A2306FC39031D0534291700349F
:1004D000A70140302602031C0800A61B08002714B1
:1004E0002230A5000800A711271C682A0830260220
:1004F000031C532A12302602031C872A16302602B8
:10050000031C532A283026020318682A0314A30D5B
:10051000A20DA10DA00DA40D2508123A031D922ACB
:10052000A9114F212508093A031DA92AA01CB92A9F
:10053000221CB92AA717200C210CCF00230603196F
:10054000AF2A4F08FF3A2306031D532A2308FF3A18
:10055000B02A25081A3A031DB92A221CB92A2308F1
:1005600030067F390319B82A23083E3A031DB92AF9
:10057000A915B114A50B0800A911A40CA00CA10C7D
:100580000318C52A2418532AC82AA717241C532A3B
:10059000A9132913200822060319D42A2008FF3A98
:1005A0002206031D532AA917210823060319DF2A4F
:1005B0002108FF3A2306FC39031D532A2917311558
:1005C0002710441D032B281021080339031DFA2A84
:1005D0004008280604390319EF2A1030C006431CCE
:1005E000F52AC41BF52A401A002B40192114401D7E
:1005F000A114032B033A0319032B401221184016B0
:100600002114A114431428114019281520093F3939
:100610000319272B21080339033A0319182BC01A91
:100620001D2B211C162B4019392B182B401D392B43
:10063000A81E1D2B5C1B9E2B5C17A71B0800200807
:100640003F39A91B403830060319BD2B0800B401FF
:100650000530B7002108FC39AC3A0319302B0800EB
:10066000FF30DF007F30DD005D08D320DD0B342B51
:100670000028A81A942BA8165C13A8134312350C53
:10068000D400540C3C39D400441F502BC41E502BB2
:10069000C31003105408103E35070318E830B500A6
:1006A000B4014312B51F431603304205D404103081
:1006B000D40203185D2B1330D4056023B700080063
:1006C00003308A00540882070634043402340234AA
:1006D0000A340634033402340E3408340534033447
:1006E00014340B34063404340E3408340434033424
:1006F00015340C34053404341B340E3407340534FB
:100700001E341234093406342B3417340B340734B6
:1007100033341A340D3408343C341E340F34093465
:100720004634213411340B34A81F992B3C08B700F0
:10073000A8135C13B401C21942131D2BA81BB12BC3
:100740001230B2000310C419B20CA81735080319EF
:1007500008000310B20C0310B20C3708BC00B7013C
:100760000800C21D1D2B3508031D1D2B4213320826
:10077000FC39103A031942171D2B401FC92BC5190C
:10078000C92B291EC62BBB202912C92B29160830BC
:10079000B30031142008C0390319D72BA10C210C48
:1007A0003F39A100201F0C2CA01B012D042E281264
:1007B000451DDC2B0430A10635080319ED2B21194A
:1007C000E72BC01FED2BA1010530B700EE2BC01B9E
:1007D000ED2BA1010530B700EE2BFF232108F839DE
:1007E000B400031DF62BC51A4213FA2BC51EFA2BB3
:1007F000421BB4013408B900A81AB4010800C0149F
:10080000211D072CC01728180A2C40110800C013FE
:100810002818052C40150800401B4A2C04308A007B
:10082000210803395424BA003A08A81EB700C2139D
:100830002119C2172C2CA81B392C4213A1194217BD
:10084000392C3108DF002330DD00D3204C08DF00D5
:100850002430DD00D320392CC01D312CA11DC01146
:10086000392CA11D392CC015421B382C4217392CAC
:100870004213C012211E422CC016C310441BC314C5
:10088000A812A813A11E0800C51D080040173908AA
:10089000B800BF28A11A0800281B502C28170800F0
:1008A00040132813B801BB288207013402340534F1
:1008B0000E34FF3FFF3FFF3FFF3FFF3FFF3FFF3F44
:1008C000FF3FFF3FFF3FFF3FFF3FFF3FFF3FFF3F38
:1008D000FF3FFF3FFF3FFF3FFF3FFF3FFF3FFF3F28
:1008E000FF3FFF3FFF3FFF3FFF3FFF3FFF3FFF3F18
:1008F000FF3FFF3FFF3FFF3FFF3FFF3FFF3FFF3F08
:10090000FF3FFF3FFF3FFF3FFF3FFF3FFF3FFF3FF7
:10091000FF3FFF3FFF3FFF3FFF3FFF3FFF3FFF3FE7
:10092000FF3FFF3FFF3FFF3FFF3FFF3FFF3FFF3FD7
:10093000FF3FFF3FFF3FFF3FFF3FFF3FFF3FFF3FC7
:10094000FF3FFF3FFF3FFF3FFF3FFF3FFF3FFF3FB7
:10095000FF3FFF3FFF3FFF3FFF3FFF3FFF3FFF3FA7
:10096000FF3FFF3FFF3FFF3FFF3FFF3FFF3FFF3F97
:10097000FF3FFF3FFF3FFF3FFF3FFF3FFF3FFF3F87
:10098000FF3FFF3FFF3FFF3FFF3FFF3FFF3FFF3F77
:10099000FF3FFF3FFF3FFF3FFF3FFF3FFF3FFF3F67
:1009A000FF3FFF3FFF3FFF3FFF3FFF3FFF3FFF3F57
:1009B000FF3FFF3FFF3FFF3FFF3FFF3FFF3FFF3F47
:1009C000FF3FFF3FFF3FFF3FFF3FFF3FFF3FFF3F37
:1009D000FF3FFF3FFF3FFF3FFF3FFF3FFF3FFF3F27
:1009E000FF3FFF3FFF3FFF3FFF3FFF3FFF3FFF3F17
:1009F000FF3FFF3FFF3FFF3FFF3FFF3FFF3FFF3F07
:100A00000800A108281A072DBB0028160800BB06FD
:100A1000031D532A21083F390319532A210CAD0025
:100A2000AD0C03182D162D080839031DAD16AD1198
:100A3000AD1BAD153F30AD050C3C0318002D053046
:100A40008A000C302D028207582D5D2D622D672DF6
:100A5000002D002D002D002D002D6D2D732D792DD5
:100A60007F2D852D8B2D912D972D9C2D002D002DCB
:100A7000002D002D002DA12DA22DA72D002DAC2D78
:100A8000002D002DAD2DB22DB72D002D002D002DE8
:100A9000002D002D002D002DBD2DC92DD52DE12DB2
:100AA000002D002DED2D002D002DF22DF82DFE2D09
:100AB000C5154508DF000830CB2845114508DF0083
:100AC0000830CB2845154508DF000830CB28C51174
:100AD000C5124508DF000830CB284413C41244086F
:100AE000DF000630CB284417C4164408DF00063068
:100AF000CB284417C4124408DF000630CB2842102C
:100B0000C2104208DF000430CB284214C210420851
:100B1000DF000430CB284210C2144208DF0004304A
:100B2000CB284214C2144208DF000430CB28C4157D
:100B30004408DF000630CB28C4114408DF0006302B
:100B4000CB28002D44114408DF000630CB28441583
:100B50004408DF000630CB28302B45164508DF005F
:100B60000830CB2845124508DF000830CB28421654
:100B7000A3204208DF000430CB28C51045104212E4
:100B8000A3204508DF000830CB204208DF000430F6
:100B9000CB28C51445144212A3204508DF000830B5
:100BA000CB204208DF000430CB28C5144510421288
:100BB000A3204508DF000830CB204208DF000430C6
:100BC000CB28C51045144212A3204508DF00083089
:100BD000CB204208DF000430CB28C5164508DF00D3
:100BE0000830CB28C41044144408DF000630CB285A
:100BF000C41444144408DF000630CB28C410441049
:100C00004408DF000630CB2864002108291B403847
:100C1000281A0D2EBB00281608003B06031D532A78
:100C20003B080319532A3B08FE393E3A0319532A5D
:100C30003B08663C031C532A3B08B000DF00281227
:100C40000230CB2840105012D012C01C0800C4182B
:100C5000352E4418352E2818352EC01B322ED012B2
:100C600050163D2E5012D0163D2EC01B3A2ED016D7
:100C700050123D2E5016D0123D2E451E0800D012A7
:100C8000501E442E5012080050160800FF3FFF3F30
:100C9000FF3FFF3FFF3FFF3FFF3FFF3FFF3FFF3F64
:100CA000FF3FFF3FFF3FFF3FFF3FFF3FFF3FFF3F54
:100CB000FF3FFF3FFF3FFF3FFF3FFF3FFF3FFF3F44
:100CC000FF3FFF3FFF3FFF3FFF3FFF3FFF3FFF3F34
:020000040001F9
:04000E009C3FFF1FF5
:080000007004083D0018000027
:10E000007D00FF00FF00FF00FF00FF00FF00FF009A
:10E01000FF00FF00FF00FF00FF00FF00FF00FF0008
:10E02000FF00FF00FF00FF00FF00FF00FF00FF00F8
:10E03000FF00FF00FF00FF00FF00FF00FF00FF00E8
:10E04000FF00FF00FF00FF00FF00FF00FF00FF00D8
:10E05000FF00FF00FF00FF00FF00FF00FF00FF00C8
:10E06000FF00FF00FF00FF00FF00FF00FF00FF00B8
:10E07000FF00FF00FF00FF00FF00FF00FF00FF00A8
:10E08000FF00FF00FF00FF00FF00FF00FF00FF0098
:10E09000FF00FF00FF00FF00FF00FF00FF00FF0088
:10E0A000FF00FF00FF00FF00FF00FF00FF00FF0078
:10E0B000FF00FF00FF00FF00FF00FF00FF00FF0068
:10E0C000FF00FF00FF00FF00FF00FF00FF00FF0058
:10E0D000FF00FF00FF00FF00FF00FF00FF00FF0048
:10E0E000FF00FF00FF00FF00FF00FF00FF00FF0038
:10E0F000FF00FF00FF00FF00FF00FF00FF00FF0028
:10E10000FF00FF00FF00FF00FF00FF00FF00FF0017
:10E11000FF00FF00FF00FF00FF00FF00FF00FF0007
:10E12000FF00FF00FF00FF00FF00FF00FF00FF00F7
:10E13000FF00FF00FF00FF00FF00FF00FF00FF00E7
:10E14000FF00FF00FF00FF00FF00FF00FF00FF00D7
:10E15000FF00FF00FF00FF00FF00FF00FF00FF00C7
:10E16000FF00FF00FF00FF00FF00FF00FF00FF00B7
:10E17000FF00FF00FF00FF00FF00FF00FF00FF00A7
:10E18000FF00FF00FF00FF00FF00FF00FF00FF0097
:10E19000FF00FF00FF00FF00FF00FF00FF00FF0087
:10E1A000FF00FF00FF00FF00FF00FF00FF00FF0077
:10E1B000FF00FF00FF00FF00FF00FF00FF00FF0067
:10E1C000FF00FF00FF00FF00FF00FF00FF00FF0057
:10E1D000FF00FF00FF00FF00FF00FF00FF00FF0047
:10E1E000FF00FF00FF00FF00FF00FF00FF00FF0037
:10E1F000FF00FF00FF00FF00FF00FF00FF00FF0027
:00000001FF
